:020000040000FA
:020000000528D1
:06000A008316073081009F
:10001000013085008601831285018601051C0E28AA
:10002000013067208600851405155F2085100511B5
:1000300061208601051C242800306720860061208D
:1000400086016120931425286120013090002B2027
:100050006720860027280518372806301002031964
:100060009001900A10086720860063202B28931CBB
:10007000851405155F20931C851005111008672055
:1000800086006120860161201008672086006120BB
:1000900086016120100867208600612086016120AA
:1000A0001008672086006120860161202D280B1131
:1000B000D93081000B1D5A28910B572808000A30AF
:1000C00064283230642805309100572008008207E8
:0E00D0003F3406345B344F3466346D347D3477
:00000001FF
